:101A300020202025732020202020202000204C6FF3
:101A40006F6B696E6720666F723A2020202020201D
:101A50000020466F756E64202532642020202020EF
:101A6000202000204D6F64756C6520435055732E07
:101A70002E2E2020200020506F6C6C696E67207322
:101A8000797374656D20200020666F72206D6F641D
:101A9000756C65732E2E2E202000456E61626C6978
:101AA0006E672052656D6F746573002020202020C2
:101AB000202020202020202020202000526563614B
:101AC0006C6C696E672020202020202000507265F9
:101AD00076696F75732050726573657420003232B9
:101AE00035730033312E3020202000323235000093
:101AF000000021006400323235730000002208FC2F
:101B00000032303600000000600B540032303700E5
:101B1000000000630E10003232320000000040105E
:101B2000CC00323233204D00005A10CC0032323318
:101B3000204100005B5EEC003232370000000023E1
:101B40006AA40032333020410000667594003233BD
:101B50003020420000677788003233302043000095
:101B600068797C0032333020440000697B70003299
:101B700031300000000020000001323439204100E3
:101B800000240960013234392042000025827801A6
:101B9000323530204200004200000232353620410A
:101BA0003100344650023235362041320036490C7D
:101BB0000232353620423100354BC80232353620EC
:101BC000423200374E84023235392041000028511C
:101BD0004002323539204200002955280232353979
:101BE000204300002A591002323539204400002BCE
:101BF0005CF802323630204100003060E0023236BC
:101C0000302042000031620C0232363120410000A7
:101C10002C633802323631204200002D6720023218
:101C20003631204300002E6B08023236312044004A
:101C3000002F6EF002323636204100003272D80298
:101C4000323636204200003373B402323530204140
:101C5000000041753002323732000000005E0000A3
:101C60000432383120413100380A2804323831201A
:101C70004231003A0B2204323831204331003C0C0F
:101C80001C04323831204431003E0D160432383104
:101C900020413200390E1004323831204232003BEC
:101CA0000F0A04323831204332003D100404323828
:101CB00031204432003F10FE0432383546204100C6
:101CC0004C11F804323835462042004D12F20432ED
:101CD0003835422041004E13EC0432383542204260
:101CE000004F157C043239312041000044170C04A8
:101CF000323931204200004528A0043239322041D7
:101D00000000483A340432393220420000493B2E68
:101D100004323932204300004A3C28043239322050
:101D20004400004B3D220432393620410000643E1D
:101D30001C0432393620420000654B000432353134
:101D4000204100005C0000050000000000000000D1
:101D50000000000000000000000000000000000083
:091D60000000000000000000007A
:0B3E2A00440343000000004103470078
:10405500E4FFFE75A70F75B7835384DFF5A775B623
:104065001075A70F43842043B30175A90175B102EB
:104075000FBF00010EEF640F4E70F543B302E5B3B9
:0640850030E4FB758F041E
:01408B002212
:10468C0075A70F75A406E4F5A5F5A675F4FC75AF32
:10469C001C75D40F75D70375E10475E2C2F5A7221A
:0D49D100E4F592F593F594F59575910422A7
:10498400758922758E0C758C5D75881075C8042226
:0C49DE00AFA7E4F5A775C80CF5CA8FA7B9
:0149EA0022AA
:10487E00AFA775A70F75BA1F75BC8475E88075D183
:06488E000A75BB118FA7A3
:014894002201
:10472B00E4FE75F00BEE901AF2120FAAE493B507A4
:0B473B0003AF06220EEEB43AE97FFF48
:014746002250
:103C6900E490021FF0A3F0A3F0A3F0E4900221F086
:103C7900A3F0900221E475F001120E39900221E0BF
:103C8900B41FEFA3E0B440EA121A27EF6009E490E9
:103C9900021FF0A3F0800A90021FE475F001120ED2
:103CA90039D3900220E094F490021FE0940140BBC4
:013CB90022E8
:1026EA00E4900375F090021F120F7900000000E4D5
:1026FA007F2DFEFDFC90021F120F2CC3120EF95003
:10270A002990021F120F2074482FF582E43403F532
:10271A0083E4F090021F120F20E47B01FAF9F81209
:10272A000E9D90021F120F6D80C590021F120F7925
:10273A0000000000E47F3AFEFDFC90021F120F2CFD
:10274A00C3120EF9400302283C90021F120F209078
:10275A001AF275F00BEF120FAAEE75F00BA425838F
:10276A00F583E493900227F07BFF7A1A793090027E
:10277A0062120FE6E47F0BFEFDFC90021F120F2C83
:10278A00120EAA74EB2FF9741A3EFA7BFF900265B7
:10279A00120FE67B007A00790812114B7B007A004F
:1027AA007908900262120FE67BFF7A1A793D12438A
:1027BA0085900227E0FF12466B900223120F7900E0
:1027CA00000000E47F987E3AFDFC900223120F2C51
:1027DA00C3120EF950447B017A027928124540EF60
:1027EA00602190022AE0B41C1A900229E0FF9003AB
:1027FA0075E02448F582E43403F583EFF09003751D
:10280A00E004F0900223120F20E47B01FAF9F81297
:10281A000E9D900223120F6D80A990021F120F20A5
:10282A00E47B01FAF9F8120E9D90021F120F6D0255
:10283A00273E7BFF7A1A7951900262120FE69003C3
:10284A0075E0FF900265E4F0A3EFF07B007A00796F
:10285A000812114B7BFF7A1A7963900262120FE613
:0B286A007B007A007908124385D2142D
:012875002240
:10144B00E4900207F0A3F0F5D912405512468C1226
:10145B0049D112498412487E1249DE12477F124944
:10146B0002124192124866124A4390039EE025E015
:10147B00FF1248EE7F211249F843CE0143E680D29A
:10148B00AF123C697BFF7A1A7988900262120FE6E1
:10149B007A1A7976124385900202120F79000000B6
:1014AB00007F807E1A7D067C00900202120F2CC3F7
:1014BB00120F0F501B900202120F20EF2401FFE4BA
:1014CB003EFEE43DFDE43CFC900202120F6D80D128
:1014DB001226EA900202120F79000000007F407E74
:1014EB000D7D037C00900202120F2CC3120F0F50C4
:1014FB001B900202120F20EF2401FFE43EFEE43D9D
:10150B00FDE43CFC900202120F6D80D11246297B48
:10151B00FF7A1A79AB900262120FE67A1A799A1255
:10152B004385900202120F79000000007F407E0D70
:10153B007D037C00900202120F2CC3120F0F501B65
:10154B00900202120F20EF2401FFE43EFEE43DFD6A
:10155B00E43CFC900202120F6D80D11245E77BFF39
:10156B007A1A79CD900262120FE67A1A79BC12437D
:10157B00851243FAD21443A82043E608E4FF12472E
:10158B0063EF600612493D124A4F7F01124763EF2A
:10159B00600612492A124A4F900207E07002A3E03C
:1015AB00604590020774FFF5F0120E39900207E0C8
:1015BB007002A3E0701B53E6EF7BFF7A1A79E3907E
:1015CB000222120FE67A1A79DE123ABC43E6108039
:1015DB0016301513E4900207F0A3F09002FD120FE2
:1015EB00C6121090124A4F124303EF607453E6EF8A
:1015FB00123BC4EF12106A163801163302162E0472
:10160B0016290816430916510A161B1000001660FE
:10161B00C21590020774FDF0A374E8F080379003B5
:10162B003C800D90033780089002F78003900334C1
:10163B00120FC6121090801D9002FA120FC68982EB
:10164B008A837F01800C9002FA120FC689828A83EB
:10165B007FFF12109443E610124303EF708F0217B3
:10166B005F7B017A027909124540EF70030217651F
:10167B0090020BE024F7700302170724FA700302A1
:10168B00171D24FC601E24FE6069241270D37D019B
:10169B007FFE124A6690020AE0FF12472B90020669
:1016AB00EFF080BD7B017A027909900219120FE6E7
:1016BB00900001120DB6FF12472B900206EFF0E0DF
:1016CB0075F00BA424EBF9741A35F0FA7BFFC00309
:1016DB00C002C001900219120FC6E92403F9E43AC3
:1016EB00FA900222120FE6D001D002D003123ABCBC
:1016FB0002166C1246291245E702166C90020BE09B
:10170B00640A700302166C7B017A02790912454058
:10171B0080EA7B017A02790990021C120FE6900095
:10172B0003120DB664C0600302166C90021C120FFC
:10173B00C6900004120DB6FF90039FE06F6003028A
:10174B00166C900005120DB6FFC3941E40030216D3
:10175B006C124A71124A4F02166C20140302158741
:10176B00900343120F387BA07A8679017800C3125D
:10177B000F0F6003021587124A4F900343120F7924
:09178B0000000000C214021587E1
:031A1200023D078B
:103D0700C0E0C0F0C083C082C0D075D000C000C082
:103D170001C002C003C004C005C006C007C2CF90DF
:103D27000347E004F0B40208124AC0900347E4F0E6
:103D3700D007D006D005D004D003D002D001D000E0
:0B3D4700D0D0D082D083D0F0D0E0328A
:10458400A2AFE433FCC2AF758F0175B7A575B7F15F
:104594008F828E83EDF0E4F58FAF04EF24FF92AFAA
:0145A40022F4
:1046AC00A2AFE433FDC2AF758F0375B7A575B7F133
:0F46BC008F828E83E4F0F58FAF05EF24FF92AF6E
:0146CB0022CC
:103E6F00900250EEF0A3EFF0A3ECF0A3EDF0EB4ACD
:103E7F006031900250E0FEA3E0FFA3E0FCA3E0F569
:103E8F00828C83E0FD124584EB1B70011A90025265
:103E9F00E475F001120E39900250E475F001120E24
:043EAF003980CB2269
:081A0A00E4900000F0A3F022BB
:1043D400900000E0FEA3E0FF1246AC900000E0FE77
:1043E400A3E0FF7C007D027B007A02123E6FE49022
:0643F4000000F0A3F0221E
:0A36D200A90590024AEEF0A3EFF004
:1036DC00EE54FEFE900000E0FCA3E0FD7002EE6CE8
:1036EC006057ED4C60031243D490024AE0FEEE5456
:1036FC00FEFE7F00900000F0A3EFF090024CEEF085
:10370C00A3EFF0A37400F0A37402F07E0290024CBD
:10371C00E475F001120E4F85F082F583E493FD9071
:10372C00024EE475F001120E4F85F082F583EDF038
:10373C00EF1F70011EEF4E70D490024AE0FCA3E024
:10374C00FDEC5401FC74022DF58274003CF583E908
:01375C00F07C
:01375D002249
:103FA800900243EEF0A3EFF0A3120FE690024874DC
:103FB800FFF5F0120E4F45F06020900243E475F0D3
:103FC80001120E4FAFF0FE900245E475F001120F9A
:0B3FD800CF120D9DFD1236D280D222C8
:103E35004202EE000042029900004202940000C1D5
:053E45000CC10BC10AD5
:0A4A7C00C20BC20CE4900298F02275
:1044D800E49002EEF0A3F0900299F0A3F0A3F0901C
:1044E8000294F0A3F090028FF0A37440F0E49002DD
:0344F80097F02218
:061A1B00124A7C0244D8CF
:0D49EB0075C19043E6019002967401F02220
:0D49F800AE071249EB900293EEF0021A1B7D
:10444600E490026AF0A3F0300B02FF22200CFDD2AA
:104456000B900291E4F0A37410F09002DCEFF0E40C
:04446600A3F07F013F
:01446A00222F
:10416200300B0A900291E07002A3E070037F0022FC
:1041720090029174FFF5F0120E399002DDE0FE0418
:10418200F074DE2EF582E43402F583EFF07F012233
:0B4A5B00300B07C20BD20C124A86225F
:0A4A8600E5C120E5FBC2C4D2C52241
:10384800900264120FE6900296E07002FF22900246
:1038580067E0FE6005D3941040037F0022124446BF
:03386800EF6049C5
:10386B00E4900269F0900267E0FF900269E0FEC30A
:10387B009F501F900264120FC68E82758300120D2B
:10388B00B6FF124162EF7002FF22900269E004F072
:10389B0080D3E4900298F0124A5B900268E07003C8
:0938AB00200CFD900298E0FF22C0
:0338B4007FFF2271
:0B306E0090025C120FE690025FEDF094
:10307900E4FFD39002EFE094009002EEE0648094C4
:103089008050012253E6FE900294E0FEA3E0249BC7
:10309900F58274023EF583E0FF900294E475F00135
:1030A900120E39FCE5F064404C7006900294F0A3CE
:1030B900F090028FE475F001120E39E4FE90025F80
:1030C900E0FDEEC39D504BEEC39F5046900294E045
:1030D900FCA3E0249BF58274023CF583E0FD900299
:1030E9005C120FC68E82758300ED120E1790029442
:1030F900E475F001120E39FCE5F064404C7006905D
:103109000294F0A3F090028FE475F001120E390ECB
:1031190080ABEEC39F5025900294E475F001120E26
:1031290039FCE5F064404C7006900294F0A3F090ED
:10313900028FE475F001120E390E80D69002EE74FA
:10314900FFF5F0120E3943E60190025FE0FEEFC38E
:073159009E50028002AF0648
:01316000224C
:10483600D39002EFE094009002EEE0648094804012
:08484600047F0180027F0022C3
:031A180002255A4A
:10255A00C0E0C0F0C083C082C0D075D000C000C047
:03256A0006C007A1
:10256D00C209E5C054FE12106A26470826470A26FE
:10257D00100C26100E26B71026B71226162226216D
:10258D002826212A26162C26162E2603C025BCC247
:10259D0025A7E025A7E2000026C2C20A9002DCE0D2
:1025AD00F5C2C2C5C2C49002DB74FFF00226C4900E
:1025BD0002DBE0FFB4FF129002DDE0F5C2C2C5C23E
:1025CD00C49002DBE4F00226C49002DDE0FEEFC30E
:1025DD009E50179002DBE0FF04F074DE2FF582E4CD
:1025ED003402F583E0F5C20226C4D2C4900298E409
:1025FD00F0C20C0226C490029874FDF0D2C5C2C47C
:10260D000226C49002DB74FFF0D20AC2C4C2C1D24A
:10261D00C50226C4E5C26007900293E0B5C20E90D4
:10262D00028EE4F0C2C5C2C4D2C10226C4C2C4C265
:10263D00C1300A028079C2C5807D90028EE0702083
:10264D00E5C2F0E0FFC3900290E09F7480F8900225
:10265D008FE064809850031244D890028EE004F00D
:10266D0090028F74FFF5F0120E39900299E0FEA3DF
:10267D00E0249BF58274023EF583E5C2F090029949
:10268D00E475F001120E39FEE5F064404E700690CF
:10269D000299F0A3F090028EE014F070099002EE12
:1026AD0075F001120E39D2C1800DC2C4300A08C2B4
:1026BD000AD2C58002D20930091053C17F43C180AF
:0C26CD00C2C5C2C4C2C1C209C20CC2C056
:1026D900D007D006D000D0D0D082D083D0F0D0E0BF
:0126E90032BE
:051A2700E5C15420FFA1
:011A2C002297
:084AA20023243230304550534B
:074AAA0043C14053E6FE2268
:102B250090024DE0FFA3E0FCA3E0FDA3120FC690C9
:102B3500025CE519F0E51AA3F0900255E090025EFB
:012B4500F09F
:0F2B4600900256EFF0A3ECF0A3EDF0A3120FE610
:102B550090025F7403F0A374E8F0E5C120E5FBD2B1
:102B6500C1C2C4D2C5E4FF9003BBF030C0FDE5C0CF
:102B750054FEFE24407003022C0B24FE602324E245
:102B8500600924FE600524E2022C13C2C5EF600330
:102B9500022C19900256E025E044A0F5C27F03807F
:102BA50073EFB4030A900257E0F5C27F058065EF25
:102BB500B4050B900257A3E0F5C27F068056EF647B
:102BC50006703190025EE0900259700875F00112AE
:102BD5000FCF8003120FC6120D9DF5C290025C74D3
:102BE500FFF5F0120E3990025CE07002A3E070244C
:102BF5007F078020EFB40706D2C47F0980169003B3
:102C0500BB7405F0800E9003BB7402F08006900340
:102C1500BB7401F0EFB40904C2C080369003BBE079
:102C2500FE64066012EEB4021690025F74FFF5F0C2
:102C3500120E3945F06008D2C5E49003BBF0FF9051
:102C450003BBE06008C2C5D2C4C2C08005C2C002D1
:072C55002B70E5C120E5FB37
:012C5C002255
:0F29EA0090024BEFF0A3ECF0A3EDF0A3120FE679
:1029F9009002537403F0A374E8F0E5C120E5FBD21B
:102A0900C1C2C4D2C5E4FF9003BBF030C0FDE5C02C
:102A190054FEFE12106A2A38002ACB382A9C8A2AC8
:102A2900D3C02A65C22A3BE02A3BE200002A3802C9
:102A39002ADBC2C5EF700F90024BE025E044A0F5F8
:102A4900C27F03022AE1EF64016003022AE19002D6
:102A59004BE025E044A1F5C27F04807CEFB4030A72
:102A690090024CE0F5C27F05806EEFB4050B900231
:102A79004CA3E0F5C27F06805FEFB40606D2C57F9E
:102A8900018055EFB404047F02804D9003BB7405A7
:102A9900F0804590024EE475F001120FCFE5C212A5
:102AA9000E0590025174FFF5F0120E39900251E0B3
:102AB9007002A3E070087F09C2C1D2C4801A7F02E4
:102AC90080169003BB7406F0800E9003BB7402F06D
:102AD90080069003BB7401F0EFB40904C2C08036CC
:102AE9009003BBE0FE64066012EEB4021690025336
:102AF90074FFF5F0120E3945F06008D2C5E4900371
:102B0900BBF0FF9003BBE06008C2C5D2C4C2C0805D
:0B2B190005C2C0022A14E5C120E5FB44
:012B2400228E
:102F780090024DEFF0900250120FE690024EECF0E6
:032F8800A3EDF0C6
:102F8B00751B00543FF51C543F6059C37440951C8E
:102F9B00FFE4951BFE900253E0FCA3E0FDC39FEC06
:102FAB009E50068C198D1A80048E198F1A122B25A0
:102FBB009003BBE060037F022290024EE519851A55
:102FCB00F0120E39900255E0700B900251E5198505
:102FDB001AF0120E39C3900254E0951AF090025376
:102FEB00E09519F0900253E0F519A3E0F51AD3E53B
:102FFB001A9400E51994004067E51A9440E519947A
:10300B00005013122B259003BBE060037F0222E4D8
:10301B00F519F51A80D890024DE0FFA3E0FCA3E070
:10302B00FDA3120FC690025CE4F07440122B3C908F
:10303B0003BBE060037F022274C0251AF51A74FFEC
:10304B003519F51990024EE475F040120E399002C5
:10305B0055E0709A90025175F040120E39022FF91B
:02306B007F00E4
:01306D002240
:104804007B017A027928E4FDFCFF1248959003BBF2
:08481400E060037F00227F0237
:01481C002279
:10398E007B017A0379AD900246120FE6E490024570
:10399E00F0900245E0FFC3940E501FEFFD7C00A394
:1039AE00E475F001120FCFE4FF124895EF60037F2C
:1039BE000122900245E004F080D7E4900245F09099
:1039CE000245E0FF904AA293FE74AD2FF582E434D7
:1039DE0003F583E06E60037F0122900245E004F060
:0639EE00E0B408DB7F03DA
:0139F40022B0
:10316100E4900227F0124804EF7002FF22904AA275
:10317100E4939003ADF0904AA3E4939003AEF090F2
:103181004AA4E4939003AFF0904AA5E4939003B06E
:10319100F0904AA6E4939003B1F0904AA7E493908B
:1031A10003B2F0904AA8E4939003B3F0904AA9E4E3
:1031B100939003B4F0A37407F0A37480F0A3E4F038
:1031C100A37402F07B017A0379AD90024BE4F0A382
:1031D100740EF0E4FDFCFF1247EAEF60037F00226A
:1031E10012398EEF640360037F01227F0E7E007D22
:1031F1000E7C007B017A027927C3E49F900254F090
:1032010074809E900253F09002557401F0E4FF1215
:103211002F789002267401F0900226E0FFC39407F4
:103221005025EF640360187B017A027927900253DD
:103231007480F0A3E4F0A304F0E4FDFC122F789075
:093241000226E004F080D17F03B5
:01324A002261
:10489500900251E4F0A304F01229EA9003BBE06012
:0748A500037F01227F0022C6
:1047D0009003CBEBF07B017A0379CB900253E4F0AA
:0A47E000A304F0E4A3F0122F7822E6
:10451E00C007900249E0FFA3E0900251CFF0A3EF55
:10452E00F0D0071229EA9003BBE060037F01227FDF
:02453E00002259
:1047EA00C00790024BE0FFA3E0900253CFF0A3EF83
:0A47FA00F0E4A3F0D007122F78229C
:0B3EB30090025D120FE6900260EDF03F
:103EBE00E4900262F090025D120FC6900260E090F4
:103ECE000267F0900261E0900268F0E4FF12384859
:103EDE00EFB4FF0D900262E0FE04F0EEC3940340D7
:033EEE00D47E007F
:013EF10022AE
:06454000900259120FE683
:104546007E007F007D10121096900259120FC67DD4
:0B4556001012306EEF7002FF227F0198
:014561002237
:104994000001FF00FF000001010000FF00FF010013
:0537D60090028AEFF0F3
:1037DB00E5682401FFE43567FAA9077B01A3120F03
:1037EB00E690028B120FC674019003986B7008E978
:1037FB0065827003EA6583700C7B017A037978909C
:10380B00028B120FE690028B120FC6E569856A8355
:10381B00856B826B7008E965827003EA6583601CB7
:10382B0090028AE0856882856783F090028B120F85
:0C383B00C6AF018A678F6890028AE0F037
:01384700225E
:103BC40053E6EFAA67A9687B01E569856A83856B7B
:103BD400826401700AE56865827004E56765837034
:103BE40003FF802B7869E475F001120FB6120D9D66
:103BF400FF74019003986569700AE56B658270042F
:103C0400E56A65837009756901756A03756B7843A4
:023C1400E610B8
:013C1600228B
:1043030053E6EFE569856A83856B826401700AE58C
:104313006865827004E56765837003FF800AAB6993
:0B432300AA6AA96B120D9DFF43E61073
:01432E00226C
:031A2400022C5D34
:102C5D00C0E0C083C082C0D075D000C001C002C02A
:0D2C6D0003C005C006C00720DF03022D05CF
:102C7A00E590541FF565656F6019E59030E402D25E
:102C8A0015E565656F900287F0541F6003756D0343
:102C9A0085656FE56D6062156DE56D705CE56E6565
:102CAA0065900287F030E00AE56520E0057F0112B1
:102CBA0037D6900287E030E10AE56520E1057F0218
:102CCA001237D6900287E030E20AE56520E2057FF6
:102CDA00041237D6900287E030E30AE56520E3055F
:102CEA007F081237D6900287E030E40AE56520E4CF
:0B2CFA00057F101237D685656EC2DF23
:062D050020D80330D95D67
:102D0B00900287E580F0C2D9C2D8E0FF656C54C051
:102D1B00604BEFC4131354037E005403FFE56CC4E4
:102D2B00540CFDED4F2494F582EE3449F583E49376
:102D3B00FF900288F0A3E566F0EF2566F566E06587
:102D4B006630E113200E10900288E0B401047F0975
:0D2D5B0080027F0A1237D6900287E0F56CE7
:102D6800D007D006D005D003D002D001D0D0D08271
:052D7800D083D0E03221
:0F49B40043E60875DA3175DB3175D983D2DE221F
:10477F001249B47B017A0379788B698A6A896B8ACB
:0B478F00678968E4900377F002456240
:10456200900377E0FF30E104C2958002D295EF30EC
:10457200E204C2968002D296EF30E303C29722D2BF
:0245820097227E
:031A2D000241C1B2
:0841C100C0E0C083C082C0D041
:1041C900900376E004F0E0B41910A3E030E004B203
:0D41D900838002D283900376E4F053913F7F
:0941E600D0D0D082D083D0E032A9
:0B4A6600900377E05FF04DF002456226
:102D7D00008040C020A060E0109050D030B070F0C6
:102D8D00088848C828A868E8189858D838B878F836
:102D9D00048444C424A464E4149454D434B474F466
:102DAD000C8C4CCC2CAC6CEC1C9C5CDC3CBC7CFCD6
:102DBD00028242C222A262E2129252D232B272F266
:102DCD000A8A4ACA2AAA6AEA1A9A5ADA3ABA7AFAD6
:102DDD00068646C626A666E6169656D636B676F606
:102DED000E8E4ECE2EAE6EEE1E9E5EDE3EBE7EFE76
:102DFD00018141C121A161E1119151D131B171F136
:102E0D00098949C929A969E9199959D939B979F9A5
:102E1D00058545C525A565E5159555D535B575F5D5
:102E2D000D8D4DCD2DAD6DED1D9D5DDD3DBD7DFD45
:102E3D00038343C323A363E3139353D333B373F3D5
:102E4D000B8B4BCB2BAB6BEB1B9B5BDB3BBB7BFB45
:102E5D00078747C727A767E7179757D737B777F775
:102E6D000F8F4FCF2FAF6FEF1F9F5FDF3FBF7FFFE5
:011A150022AE
:1048EE00EF30E104D2818002C281EF30E203D28246
:0448FE0022C282222E
:104902007F381249167F061249167D0EE4FF124ABD
:044912001F021A1551
:10491600900265EFF012484EEF20E7F9900265E04D
:04492600FF02408CC0
:10484E0075A0FFC2B3D2B4D2B27F14DFFEAFA0EF19
:07485E00902D7D93FFC2B213
:014865002230
:054AB7007F0102491619
:10408C00EF902D7D93F5A07FC87E00EF1F70011E71
:10409C00EF4E70F7C2B3C2B4D2B27E007FC8EF1F2E
:1040AC0070011EEF4E70F7C2B27E007FC8EF1F701A
:0640BC00011EEF4E70F73B
:0140C20022DB
:1040FA00EF3395E0FE747D2FF582742D3EF583E44F
:10410A0093F5A0C2B4D2B2D2B37FC87E00EF1F70BB
:10411A00011EEF4E70F7C2B27E007FC8EF1F70011A
:05412A001EEF4E70F7CE
:01412F00226D
:0C4A1F009003CCE05FF04DFFF002491660
:0E49C300AE0712484EEF20E7F9AF060240FAA9
:10446B00900265120FE6900265120FC6120D9D6049
:10447B0013900265E475F001120FCF120D9DFF1220
:05448B0049C380E2229C
:1043850090025F120FE6124AB7E4FDFF124A2B9026
:10439500025F120FC612446BE4FD7F01124A2B9097
:0843A5000262120FC602446B14
:0C4A2B00EF75F040A42D2480FF02491616
:1045A500E4900245F0A37422F0A3741DF0A374FFF8
:1045B500F07B017A027945E4900261F07D04023EC8
:0145C500B342
:1045C600E4900245F0A37422F0A3741EF0A374FFD6
:1045D600F07B017A027945E4900261F07D04023EA7
:0145E600B321
:1046CC00E4900225F0A37422F0A37401F0A3EFF0A0
:1046DC007B017A027925E4900261F07D04023EB3FD
:1046EC00E4900225F0A37422F0A37402F0A3EFF07F
:1046FC007B017A027925E4900261F07D04023EB3DD
:1045E700E4900225F0A37422F0A37416F0A374FFDD
:1045F700F07B017A027925E4900261F07D04023EA6
:01460700B3FF
:10460800E4900225F0A37422F0A37417F0A374FFBA
:10461800F07B017A027925E4900261F07D04023E84
:01462800B3DE
:10462900E490021FF0A37422F0A37414F0A374FFA2
:10463900F07B017A02791FE4900261F07D04023E69
:01464900B3BD
:10464A00E49003C4F0A37422F0A3741BF0A374FFD4
:10465A00F07B017A0379C4E4900261F07D04023EA2
:01466A00B39C
:10466B00900259EFF0A37422F0A3741AF0A374FF15
:10467B00F07B017A027959E4900261F07D04023EED
:01468B00B37B
:1041EF00E4900249F0A37422F0A37404F0A3EFF05B
:1041FF00900248E090024DF0A3EDF0A3EBF07B01AD
:0E420F007A027949E4900261F07D07023EB325
:10421D00E4900247F0A37422F0A37405F0A3EFF02D
:10422D00900246E090024BF0A3EDF0A3EBF07B0182
:0E423D007A027947E4900261F07D07023EB3F9
:10424B00E4900234F0A37422F0A37407F0A3EFF010
:10425B00A3EDF0A3EBF0900233E090023AF07B0178
:0E426B007A027934E4900261F07D07023EB3DE
:10427900E4900234F0A37422F0A37408F0A3EFF0E1
:10428900A3EDF0A3EBF0900233E090023AF07B014A
:0E4299007A027934E4900261F07D07023EB3B0
:1039250020202020496E76616C69642020202020AB
:10393500002000202020202020446F6E65202020BC
:103945002020004E6F7420526573706F6E64696E2F
:10395500672E2E2E00202020202020202020202011
:1039650000437264204E6F7420466F726D617474EB
:103975006400466F72205072657365747300202071
:0939850020202020202020200039
:10470C00121A0A7E607F027B017A03799E9002481E
:0F471C00E4F0A37402F0123FA81243D4C210229B
:10346B009002207403F0E4A3F0A3F090039E04F009
:10347B00A3740FF012470C121A0A7E607F017B01B6
:10348B007A027920900248E4F0A304F0123FA87E60
:10349B00007F0D7D007B007A00794B121096E49033
:1034AB00021FF090021FE0FFC3941E502875F00D11
:1034BB00EF906004120FAAAF82AE837B007A007983
:1034CB004B900248E4F0A3740DF0123FA890021F3A
:1034DB00E004F080CE7E607F007B017A0279219040
:1034EB000248E4F0A304F0123FA87E617F8A7B01BF
:1034FB007A027922900248E4F0A304F0123FA8026A
:02350B0043D4A7
:10419200906000E493F46007A3E493640360031265
:1041A200346B789E7C037D017BFF7A6079027E000E
:0F41B2007F02120D77E4900399F0900398F022AA
:103CBA00900398E0FFC3941E5042A3E0C3941E50A1
:103CCA003BEF75F00DA42404F9746035F0FA7BFF1C
:103CDA00784B7C007D007E007F0D120D7790039952
:103CEA00E075F00DA42404F9746035F0FA7BFF78CE
:0D3CFA00587C007D007E007F0D120D7722AA
:103FE300900225120FE6900399E0C3941E50291204
:103FF3001A0A900399E075F00D906004120FAAAFAE
:1040030082AE83900225120FC6900248E4F0A37497
:094013000DF0123FA81243D42263
:094A90007B007A007958023FE333
:10432F00301122900398E075F00DA42404F9746005
:10433F0035F0FA7BFF784B7C007D007E007F0D12FD
:0C434F000D77124A9030100312470C2228
:1043FA0090618AE493FFC3941E5009900399EFF0E9
:10440A00900398F0900398E0FF1246CC123CBAE46D
:06441A00FD7FFE024A6670
:10413000900399E0900398F0E0FF1246CC123CBA4D
:10414000E4FD7FFE124A66121A0A7E617F8A7B01B5
:104150007A037998900248E4F0A304F0123FA80291
:0241600043D446
:10479A007B007A00794B123FE3123CBA900399E00E
:0B47AA00FF1246ECE4FD7FFE024A66B1
:0B4A7100900399EFF0123CBA024130B4
:10493D00900399E004F0E0B41E02E4F0123CBA02D8
:02494D004130F7
:10492A00900399E014F0E0B4FF03741DF0123CBA4E
:03493A0002413007
:0F2E7D00900226EDF0900225EFF0900227EBF087
:102E8C00B5070E900226E0FF900228E0B5070280FD
:102E9C002B900227E0FF900225E0C39F5009A3E08E
:102EAC00FEEF9E50028015900227E0FF900225E075
:102EBC00FED39F401A900228E09E40137BFF7A3984
:102ECC00793690025C120FE67A397925022F7490CC
:102EDC000225E0FFA3E0FDA3E0FBA3E0900233F0AA
:102EEC0012424B900225E0900229F0900227E090CC
:102EFC00022AF0900226E0FF900229E0FED39F50B8
:102F0C005175F00DEE906004120FAAAF82AE839053
:102F1C00022EEEF0FCA3EFF0FD90022AE075F00D0E
:102F2C00906004120FAAAA83A9827BFF90022B1235
:102F3C000FE6AE02AF01AA04A905900248E4F0A383
:102F4C00740DF0123FA8900229E004F0A3E004F005
:102F5C0080A11243D4123CBA7BFF7A3979369002A5
:0B2F6C005C120FE67A397938123DE460
:012F77002237
:0F287600900226EDF0900225EFF0900227EBF094
:10288500B5070E900226E0FF900228E0B50702800A
:102895002B900227E0FF900225E0C39F5009A3E09B
:1028A500FEEF9E50028015900227E0FF900225E082
:1028B500FED39F401A900228E09E40137BFF7A3991
:1028C500793690025C120FE67A3979250229E6906D
:1028D5000225E0FFA3E0FDA3E0FBA3E0900233F0B7
:1028E500124279900225E0900229F0900227E090AB
:1028F500022AF0900226E0FF900229E0D39F4003D0
:102905000229D3A3E075F00D906004120FAAAA83E3
:10291500A9827BFF90022B120FE6E4FFFE90022BAB
:10292500120FC6120D9DFD74A02FF58274033EF59E
:1029350083EDF090022CE475F001120E390FBF0003
:10294500010EEF640D4E70D5900229E075F00D90E3
:102955006004120FAAAF82AE8390022EEEF0FCA3A4
:10296500EFF0FD90022AE075F00D906004120FAAB9
:10297500AA83A9827BFF90022B120FE6AE02AF015C
:10298500AA04A905900248E4F0A3740DF0123FA82B
:102995001243D4900229E075F00D906004120FAA3D
:1029A500AF82AE8390022EEEF0A3EFF07B017A03A7
:1029B50079A0900248E4F0A3740DF0123FA81243E9
:1029C500D4900229E004F0A3E004F00228F8123CB8
:1029D500BA7BFF7A39793690025C120FE67A39793B
:0429E50038123DE483
:0129E90022CB
:1023A600E4900248F0900247F0900375E0FF900237
:1023B60047E0FEC39F400302254A74482EF582E497
:1023C6003403F583E0FF12466B90039A120F7900EF
:1023D6000000007B017A027949124540EF601090B7
:1023E600024BE0B41C09900248E004F00225179065
:1023F600039A120F20E47B01FAF9F8120E9D90035E
:102406009A120F6D7F407E427D0F7C0090039A12D8
:102416000F2CC3120EF970BB900247E075F00BA4A7
:1024260024EBF9741A35F0FA7BFFC002C0017A3941
:10243600794890025C120FE6D001D002123DE4E426
:10244600900245F0A3F0900245E0FEA3E0FFE4FC15
:10245600FD7B607AEAF9F8D3120EF9400C9002453A
:10246600E475F001120E3980DDE4900245F0A3F028
:10247600900245E0FEA3E0FFE4FCFD7B607AEAF90A
:10248600F8D3120EF9400C900245E475F001120ED5
:102496003980DDE4900245F0A3F0900245E0FEA30A
:1024A600E0FFE4FCFD7B607AEAF9F8D3120EF9400E
:1024B6000C900245E475F001120E3980DDE49002BD
:1024C60045F0A3F0900245E0FEA3E0FFE4FCFD7BAF
:1024D600607AEAF9F8D3120EF9400C900245E475D9
:1024E600F001120E3980DDE4900245F0A3F090026F
:1024F60045E0FEA3E0FFE4FCFD7B607AEAF9F8D351
:10250600120EF9400C900245E475F001120E398066
:10251600DDE4900245F0A3F0900245E0FEA3E0FF63
:10252600E4FCFD7B607AEAF9F8D3120EF9400C90D0
:102536000245E475F001120E3980DD900247E00491
:10254600F00223AF900375E0FF900248E06F60034E
:032556000223A6B7
:01255900225F
:10209400E490022CF0A2AF33900231F0124AAA125B
:1020A400398E900244EFF07F221249F8900244E006
:1020B400640360030223927BFF7A39795A7F031207
:1020C40033C01245A51223A6E4900226F0900375AE
:1020D400E0FF900226E0FEC39F40030222C674483C
:1020E4002EF582E43403F583E0FF90022AF01247D0
:1020F4002B90022BEFF0E075F00BA424EBF9741A8B
:1021040035F0FA7BFF7F031233C090022BE0FC759D
:10211400F00B901AF3120FAAE493FE740193FDEEF0
:10212400FB75F00BEC901AF5120FAAE49390024899
:10213400F090022AE0FF1241EF90039A120F790007
:102144000000007B017A027934124540EF601E9052
:102154000236E0B40A177B017A0279349000031244
:102164000DB6FF90022AE06F700302229390039A47
:10217400120F20E47B01FAF9F8120E9D90039A12D3
:102184000F6D7F407E427D0F7C0090039A120F2CCE
:10219400C3120EF970AD90022BE075F00BA424EB82
:1021A400F9741A35F0FA7BFFC002C0017A39794814
:1021B40090025C120FE6D001D002123DE4E49002DA
:1021C40027F0A3F0900227E0FEA3E0FFE4FCFD7BF0
:1021D400607AEAF9F8D3120EF9400C900227E475FC
:1021E400F001120E3980DDE4900227F0A3F0900292
:1021F40027E0FEA3E0FFE4FCFD7B607AEAF9F8D374
:10220400120EF9400C900227E475F001120E398089
:10221400DDE4900227F0A3F0900227E0FEA3E0FFA4
:10222400E4FCFD7B607AEAF9F8D3120EF9400C90D5
:102234000227E475F001120E3980DDE4900227F0E4
:10224400A3F0900227E0FEA3E0FFE4FCFD7B607AAC
:10225400EAF9F8D3120EF9400C900227E475F00164
:10226400120E3980DDE4900227F0A3F0900227E0FB
:10227400FEA3E0FFE4FCFD7B607AEAF9F8D3120EDA
:10228400F9400C900227E475F001120E3980DDE468
:10229400900227F0A3F0900227E0FEA3E0FFE4FC05
:1022A400FD7B607AEAF9F8D3120EF9400C9002270C
:1022B400E475F001120E3980DD900226E004F0028C
:1022C40020D1C2AF124AAA7F2212472B90022BEFD1
:1022D400F0E0FF75F00B901AF5120FAAE493FD904D
:1022E400022DE4F0A3EDF075F00BEF901AF3120F4A
:1022F400AAE493FF74019390022FCFF0A3EFF09020
:10230400022BE075F00BA424EBF9741A35F0FA7B78
:10231400FF7F031233C0E4900229F0900229E0FF0A
:10232400C3941E504675F00DEF906004120FAAAFCF
:1023340082AE83900232EEF0FAA3EFF0FB90022D0E
:10234400A3E0FFA3E0FCA3E0FDA9037BFF90024B05
:10235400E4F0A3740DF01247EA90022FE475F00D37
:10236400120E39900229E004F080B07F221249F85D
:10237400900231E024FF92AF7BFF7A3979369002E4
:102384005C120FE67A397938123DE40245C67BFFC8
:102394007A39797790025C120FE67A397966123DC0
:0123A400E454
:0123A5002215
:101D6900A2AFE43390022FF0124AAA12398E9002E0
:101D790042EFF07F221249F8900242E064036003C7
:101D89000220807BFF7A3979837F021233C01245A2
:101D9900A51223A6E4900225F0900375E0FF9002B6
:101DA90025E0FEC39F4003021F9774482EF582E485
:101DB9003403F583E0FF900229F012472B90022AA1
:101DC900EFF0E075F00BA424EBF9741A35F0FA7B07
:101DD900FF7F021233C090022AE0FC75F00B901AC3
:101DE900F3120FAAE493FE740193FDEEFB75F00B59
:101DF900EC901AF5120FAAE493900246F09002298A
:101E0900E0FF12421D90039A120F79000000007B37
:101E1900017A027932124540EF601E900234E0B433
:101E29000A177B017A027932900003120DB6FF90EE
:101E39000229E06F7003021F6490039A120F20E4D5
:101E49007B01FAF9F8120E9D90039A120F6D7F40EB
:101E59007E427D0F7C0090039A120F2CC3120EF95B
:101E690070AD90022AE075F00BA424EBF9741A35D1
:101E7900F0FA7BFFC002C0017A39794890025C12FE
:101E89000FE6D001D002123DE4E4900226F0A3F05F
:101E9900900226E0FEA3E0FFE4FCFD7B607AEAF90C
:101EA900F8D3120EF9400C900226E475F001120ED7
:101EB9003980DDE4900226F0A3F0900226E0FEA32B
:101EC900E0FFE4FCFD7B607AEAF9F8D3120EF940F1
:101ED9000C900226E475F001120E3980DDE49002BF
:101EE90026F0A3F0900226E0FEA3E0FFE4FCFD7BD0
:101EF900607AEAF9F8D3120EF9400C900226E475DB
:101F0900F001120E3980DDE4900226F0A3F0900270
:101F190026E0FEA3E0FFE4FCFD7B607AEAF9F8D352
:101F2900120EF9400C900226E475F001120E398068
:101F3900DDE4900226F0A3F0900226E0FEA3E0FF84
:101F4900E4FCFD7B607AEAF9F8D3120EF9400C90B3
:101F59000226E475F001120E3980DDE4900226F0C4
:101F6900A3F0900226E0FEA3E0FFE4FCFD7B507A9B
:101F7900C3F9F8D3120EF9400C900226E475F0016A
:101F8900120E3980DD900225E004F0021DA2C2AFD5
:101F9900124AAA7F2212472B90022AEFF0E0FF751E
:101FA900F00B901AF5120FAAE493FD90022BE4F0BE
:101FB900A3EDF075F00BEF901AF3120FAAE493FF5B
:101FC90074019390022DCFF0A3EFF090022AE075EF
:101FD900F00BA424EBF9741A35F0FA7BFF7F021297
:101FE90033C0E4900228F090022BA3E0FFA3E0FCA9
:101FF900A3E0FD7B017A0379A0900249E4F0A37480
:102009000DF012451E90022DE475F00D120E399057
:102019000228E075F00D906004120FAAAF82AE831A
:10202900900230EEF0A3EFF0121A0A900230E0FEAF
:10203900A3E0FF7B017A0379A0900248E4F0A3743E
:102049000DF0123FA81243D4900228E004F0E0C337
:10205900941E40937F221249F890022FE024FF92A8
:10206900AF7BFF7A39793690025C120FE67A3979BB
:1020790038123DE40245C67BFF7A39797790025CD4
:0A208900120FE67A397966123DE481
:01209300222A
:10179400205072696D6F2056657273696F6E2000F8
:1017A40020496E697469616C697A696E67202020CA
:1017B4000025326420006F6666006F6E0052656D0E
:1017C4006F74650042617365204368616E6E656C79
:1017D4003A2025326400456E61626C656400446998
:1017E4007361626C65640053746174757300466F51
:1017F400726D617474696E672043617264000041A4
:10180400726520796F7520737572653F2020200002
:101814006C6173742F4E4F206E6578742F59455345
:1018240000202020204E6F2043617264202020205D
:10183400002000202020202020446F6E65202020DE
:101844002020004469737020436F6E747261737456
:101854003A20256400466F726D617420436172649E
:101864002020202020004D6F64756C6520257300B6
:101874004669726D776172652025730050726573D5
:101884006574204D6F646966696564002020205288
:101894006573746F72696E672020200020202042D7
:1018A40061636B696E672055702020002020202022
:1018B400436F7079696E6720202020002020204526
:1018C400786368616E67696E67202020200020209D
:1018D400204D6F64756C652025732020200025320F
:1018E400642D2532643A2532642D25326400436F19
:1018F40070792045786368616E676500526573741A
:101904006F72652066726F6D20437264004261637A
:101914006B757020746F20436172640020414243F0
:101924004445464748494A4B4C4D4E4F50515253FB
:101934005455565758595A616263646566676869B5
:101944006A6B6C6D6E6F707172737475767778797B
:101954007A303132333435363738397E21402324D6
:10196400255E262A28292D2B3D7C0102F2442001E4
:1019740002FD49730102FA47470102F741300103AE
:1019840034479A010337492A01033C493D000000CA
:1019940000000102F2481D0102FD401C0103374A08
:1019A4009901033C4A050102FA3F6C000000000063
:1019B4000102F2324B0102FD4A4301033747B501EC
:1019C400033C48AC0000000000FF17BAFF17BE003C
:1019D40007FF4A12010FFF4A37000FFF48C20100F8
:1019E400FF3B1A0001FF363C0004FF35A50007FF4A
:1019F4003A5A0100FF42D50105FF42A70000FF4902
:061A04004F0100FF4961E3
:063E4A00C10E410333002C
:10486600E4F524F5237BFF7A1779A4900262120FF0
:08487600E67A177994024385EC
:044ABC00E4F52822D3
:10375E00900225EEF0A3EFF0AF051DEF6069900229
:10376E0025E0FEA3E0F5828E83A3A3120FEFE528DA
:10377E0075F005A42402F582E43403F583120FE6F6
:10378E00900225E0FEA3E0FFF5828E83E493FCE534
:10379E002875F005A42400F582E43403F583ECF0DB
:1037AE008F828E83740193FFE52875F005A42401A2
:1037BE00F582E43403F583EFF00528900225E475D5
:0837CE00F005120E3980912272
:103D5200AB25AA26A927120D9DFE75F005A4240005
:103D6200F582E43403F583E0FFEE75F005A4240147
:103D7200F582E43403F583E0FD124A2BAB25AA2633
:103D8200A927120D9D75F005A42402F582E43403DF
:0B3D9200F583120FC69002FA020FE644
:1047B500AB25AA26A927120D9D7005E528120E0521
:0B47C500AB25AA26A92774FF020DE314
:1048AC00AB25AA26A9277401120DE3120D9DB5287C
:0648BC0004E4120E0522C7
:011A160022AD
:104490007BFF7A1A7916900334120FE69002F71216
:1044A0000FE6900337120FE690033C120FE69002DE
:0444B000FA020FE617
:103D9D00900225120FE6124490900225120FC612C2
:103DAD000FFBEA494B602F900225120FC6900003BE
:103DBD00120E65AAF0F97BFFC003C002C00190028C
:103DCD0025120FC6120FFB12101B900226E475F080
:073DDD0005120E3980C3221C
:0938B700900225EFF0A3120FE6C8
:1038C0007BFF7A1779B5900262120FE6ED2401FEB4
:1038D000E433900265F0A3CEF07B017A02792A12DC
:1038E000114B900225E0FFE4FD124A2B7B017A0286
:1038F000792A12446BE4900229F0900226E475F0D4
:1039000001120FCF120D9D90192093FF1249C39001
:103910000229E004F0E0C3940D40DF900225E0FFAF
:053920007D01024A2BAD
:10474700900399E02FF0E0FFB41E04E4F0800AEF35
:0C475700B4FF06900399741DF0023CBAF8
:103F6C00900332E0FE2458F9E4FAFBEE6014120DD3
:103F7C009D700F900332E02457F8E66005120E0591
:103F8C008004EF120DE3120D9DFFB44E04744D80AE
:0B3F9C0005EFB4FF04E4120E05D21183
:013FA70022F7
:094A9900900332E0600214F022E7
:0D4A0500900332E0C3940C5003E004F02253
:0844B4007B01AD07900229F025
:1044BC00ED120DE3120D9DFFB4FF03E4800A900290
:0C44CC0029E0FEB50705EE14120E0522D3
:0D4A1200EFB40104D20D8002C20DD20F22BC
:1048C2007A03799E74041244B490039EE025E0FFBB
:0648D2001248EED2102294
:0C4A37007A03799F74101244B4D210224C
:011A170022AC
:10401C0012432F7BFF7A35790D9002F2120FE6C214
:10402C000F7A4879D89002FD120FE67A4A791290ED
:10403C0002FA120FE67A4779B5900337120FE67A37
:09404C004879AC90033C020FE638
:1048D8007BFF7A3979F59002F2120FE67A4079C3B4
:0648E8009002FD020FE644
:104973007BFF7A197996123D9DE4900332F0C211C0
:014983002211
:0C4A430012432F7BFF7A19796E023D9D13
:10350D007D027FF3124A667BFF7A1779C1900262C2
:10351D00120FE67B007A00792912114B7BFF7A1787
:10352D0079C8900262120FE690039FE02401FEE439
:10353D0033900265F0A3CEF07B007A00793A121138
:10354D004B7B007A00793A900262120FE67A00798D
:10355D00291243857D07E4FF124A2B300F19300DD8
:10356D000B1245E77BFF7A1779DA80111246087B3B
:10357D00FF7A1779E280067BFF7A1779EB12446B9D
:10358D00124ABC7E197FD37D0212375E75250075F8
:08359D002600752723023D52B0
:103EF2007BFF7A1779F2900262120FE67B007A005A
:103F0200792912114B7BFF7A187902900262120F03
:103F1200E67B007A00793A12114B7B007A00793AFB
:0D3F2200900262120FE67A007929024385B1
:103F2F007BFF7A187903900262120FE67B007A000A
:103F3F00792912114B7BFF7A187914900262120FB4
:103F4F00E67B007A00793A12114B7B007A00793ABE
:0D3F5F00900262120FE67A00792902438574
:1044FB00123F2F124303EF60FA53E6EF123BC4EF68
:10450B0024FC600724FC70067F01227F002243E617
:03451B001080E02D
:103B1A00EF6401704F1244FBEF6049D20E123EF27D
:103B2A00124AAA123161900225EFF070137BFF7AD4
:103B3A0018793590025C120FE67A187925123DE45D
:103B4A00900225E0B403161220947BFF7A18793587
:103B5A0090025C120FE67A187937123DE47F21123F
:043B6A0049F8C20E46
:013B6E002234
:1039F5007BFF7A187947900262120FE690039EE0EA
:103A05002401FEE433900265F0A3CEF07B007A003A
:103A1500792912114B7BFF7A187959900262120F9E
:103A2500E67B007A00793A12114B7B007A00793AED
:103A3500900262120FE67A007929124385124ABC78
:103A45007E197FDD7D0212375E75250075260075AE
:053A55002724023D5290
:1049A400900399E0FD7B007A0079587F010238B7C3
:10481D007D047FF5124A66124AB71249A4900332FD
:09482D00E02403FD7F01024A2B87
:104420007D087FF9124A66124AB7900398E075F04A
:104430000DA42404F9746035F0FA7BFFE0FDE4FF7D
:064440001238B70249A486
:103ABC0090021F120FE67BFF7A18796A900262124D
:103ACC000FE690021F120FC6900265120FE67B00E4
:103ADC007A00792912114B7BFF7A18797490026263
:103AEC00120FE6900222120FC6900265120FE67BAF
:103AFC00007A00793A12114B7B007A00793A9002E5
:0E3B0C0062120FE67A007929124385D2142244
:103C17009003C8120FE67BFF7A18796A9002621246
:103C27000FE69003C8120FC6900265120FE67B00DD
:103C37007A00792912114B7BFF7A187980900262FA
:103C4700120FE67B007A00793A12114B7B007A005B
:103C5700793A900262120FE67A007929124385D2E7
:023C6700142225
:0C4A4F009002F2120FC612109002456295
:10363C00EFB4011C9002F0E07004A3E0641E900251
:10364C00F07007F0A3741EF0802DE475F001802457
:10365C00D39002F1E094019002F0E06480948040F9
:10366C001690033AE07004A3E0641E600A9002F026
:10367C0074FFF5F0120E399002F0E0FEA3E0FFC3E8
:10368C00900342E09FEE6480F8900341E0648098E0
:10369C005005EEF0A3EFF0C3900342E09FFF9003C0
:1036AC0041E09EFED3EF940EEE6480948040149023
:1036BC0002F1E0240EFE9002F0E03400900341F0A1
:0636CC00A3CEF0024A4FFC
:1035A500EFB4012B900341E07004A3E0641E700AA0
:1035B500900341F0A3741EF0804B90033AE0700431
:1035C500A3E0641E603F900341E475F001803390F1
:1035D50002F0E0FEA3E0FF900341E0FCA3E0FDB5AF
:1035E500070EECB5060A900341EEF0A3EFF0801547
:1035F500D3ED9401EC64809480400A90034174FFFC
:10360500F5F0120E399002F0E0FEA3E0FF900341C1
:10361500E0FCA3E0FDC39FFFEC9EFED3EF940EEE0E
:1036250064809480400EED24F2FEEC34FF9002F0AD
:07363500F0A3CEF0024A4FA2
:103A5A009002F0A3E0FE900341A3E0C39EFEEFB400
:103A6A00013590033FE0FCA3E0FD641E4C700A9010
:103A7A00033FF0A3741EF08036AF067E00ED2FFFE1
:103A8A00EE3CFEC3EF941EEE6480948050219003B6
:103A9A003FE475F0018015D3900340E09401900350
:103AAA003FE064809480400774FFF5F0120E3902FB
:023ABA004A4F71
:1042A700EF64017028D20E9002F0A3E014FF900390
:1042B70041A3E014FD90033FA3E014FB90033AE011
:0E42C700F8A3E014900228F0122876C20E220E
:103DE400900259120FE6900259120FC69002621205
:103DF4000FE67B007A00792912114B90025C120FB6
:103E0400C6900262120FE67B007A00793A12114BD7
:103E14007B007A00793A900262120FE67A007929DF
:063E2400124385D21422B6
:1033C000900246120FE6900245EFF0BF02157BFF18
:1033D0007A187990900262120FE67B007A007929C0
:1033E00012114B900245E0B403157BFF7A1879A0C7
:1033F000900262120FE67B007A00792912114B903D
:103400000245E0B404157BFF7A1879B0900262128D
:103410000FE67B007A00792912114B900245E0B447
:1034200005157BFF7A1879C0900262120FE67B00C7
:103430007A00792912114B7BFF7A1879D2900262B7
:10344000120FE6900246120FC6900265120FE67B3D
:10345000007A00793A12114B7B007A00793A900297
:0B34600062120FE67A00792902438512
:1042D500EF64017028D20E9002F0A3E014FF900362
:1042E50041A3E014FD90033FA3E014FB90033AE0E3
:0E42F500F8A3E014900228F0122E7DC20E22D3
:10494F00EFB4010D1244FBEF6007D20E121D69C2C6
:02495F000E2226
:10496100EFB4010D1244FBEF6007D20E122094C286
:024971000E2214
:1040C3007BFF7A32794B9002F2120FE67A43795BE7
:1040D3009002FD120FE69002F0E4F0A304F09003C7
:1040E30041E4F0A304F090033FE4F0A304F0900351
:0740F3003AE4F0A304F022FF
:10324B009002F0E0FEA3E0FF900341E0FAA3E0FB65
:10325B00C39FFFEA9EFE90033FE0FCA3E0FD2FFF20
:10326B00EC3E90033AF0A3EFF09002F0E0FEA3E007
:10327B00FFC3EB9FEE6480F8EA6480985007E490FC
:10328B00033AF0A3F07BFF7A1879E2900262120FF7
:10329B00E6900265EEF0A3EFF0900341E0FFA3E0B0
:1032AB00900267CFF0A3EFF0A3ECF0A3EDF0900347
:1032BB003AE0FFA3E090026BCFF0A3EFF07B007A34
:1032CB0000792912114B7BFF7A1879F29002621266
:1032DB000FE67B007A00793A12114B7B007A00796A
:1032EB003A900262120FE67A007929124385124A4C
:1032FB00BC7E197FE77D0512375E752501752602A9
:06330B007527F5023D529A
:10435B007BFF7A3B796F9002F2120FE67A4A794330
:10436B009002FD120FE67A4779B5900337120FE6EC
:0A437B007A4879AC90033C020FE68B
:103B6F007BFF7A197900900262120FE67B007A00D0
:103B7F00792912114B7BFF7A197911900262120F7A
:103B8F00E67B007A00793A12114B7B007A00793A82
:103B9F00900262120FE67A007929124385124ABC0D
:103BAF007E1A7F007D0212375E752501752602751C
:053BBF0027F6023D5253
:03000000020C00EF
:03000300021A03DB
:03000B00021A06D0
:03001300021A09C5
:03001B00021A0CBA
:03002300021A0FAF
:03002B00021A12A4
:03003300021A1599
:03003B00021A188E
:03004300021A1B83
:03004B00021A1E78
:03005300021A216D
:03005B00021A2462
:03006300021A2757
:03006B00021A2A4C
:03007300021A2D41
:100C0000E4F5D9E5EF7480F5FF7402F5EF787FE441
:100C1000F6D8FD9000007F007E04E4F0A3DFFCDE48
:070C2000FA75816F020C62FE
:103E50004103C0004103C2004103C1004103C3004C
:0E3E6000C113C1124203BE00004203BC0000A9
:064AB1009003C0E0FF22AB
:10476300E4FEEF14600C047010A213E433FEC213D2
:0B4773008007A212E433FEC212AF0662
:01477E002218
:044AC00043E8102295
:031A21000233117C
:10331100C0E0C0F0C083C082C0D075D000C000C280
:10332100ED9003C0E09003C2F0E5BEC4540F9003DA
:10333100C0F09003C2E0D39403501D9003C0E09409
:103341000340159003BCE07002A3E0700BD2129011
:1033510003BC04F0A374F4F09003BCE07002A3E09A
:10336100600A9003BC74FFF5F0120E399003C1E0BE
:103371009003C3F0A280E4339003C1F09003C3E053
:10338100701C9003C1E0B401159003BEE07002A36C
:10339100E0700BD2139003BE04F0A374F4F0900319
:1033A100BEE07002A3E0600A9003BE74FFF5F01264
:0F33B1000E39D000D0D0D082D083D0F0D0E0320F
:100C270002144BE493A3F8E493A34003F68001F284
:100C370008DFF48029E493A3F85407240CC8C333CE
:100C4700C4540F4420C8834004F456800146F6DF9D
:100C5700E4800B0102040810204080903E2AE47EC5
:100C6700019360BCA3FF543F30E509541FFEE49392
:100C7700A360010ECF54C025E060A840B8E493A359
:100C8700FAE493A3F8E493A3C8C582C8CAC583CA84
:100C9700F0A3C8C582C8CAC583CADFE9DEE780BE3C
:013E6E000053
:100CA700E709F608DFFA8046E709F208DFFA803E2F
:100CB70088828C83E709F0A3DFFA8032E309F6081C
:100CC700DFFA8078E309F208DFFA807088828C8384
:100CD700E309F0A3DFFA806489828A83E0A3F60838
:100CE700DFFA805889828A83E0A3F208DFFA804C12
:100CF70080D280FA80C680D4806980F280338010E9
:100D070080A680EA809A80A880DA80E280CA803351
:100D170089828A83ECFAE493A3C8C582C8CCC583C9
:100D2700CCF0A3C8C582C8CCC583CCDFE9DEE78099
:100D37000D89828A83E493A3F608DFF9ECFAA9F018
:100D4700EDFB2289828A83ECFAE0A3C8C582C8CC6E
:100D5700C583CCF0A3C8C582C8CCC583CCDFEADE87
:100D6700E880DB89828A83E493A3F208DFF980CCE9
:100D770088F0EF60010E4E60C388F0ED2402B404E2
:100D87000050B9F582EB2402B4040050AF23234589
:060D97008223900CF773AB
:100D9D00BB010689828A83E0225002E722BBFE0254
:090DAD00E32289828A83E4932287
:100DB600BB010CE58229F582E5833AF583E02250F2
:100DC60006E92582F8E622BBFE06E92582F8E2223C
:0D0DD600E58229F582E5833AF583E4932256
:100DE300BB010989828A83F8E028F022500327F7A0
:100DF30022BBFE05F8E328F3228A838982F8E49371
:020E03002822A3
:100E0500BB010689828A83F0225002F722BBFE01CC
:020E1500F322C6
:100E1700F8BB010DE58229F582E5833AF583E8F011
:100E2700225006E92582C8F622BBFE05E92582C8BD
:020E3700F222A5
:100E3900C5F0F8A3E028F0C5F0F8E5821582700244
:060E49001583E038F022E1
:100E4F00A3F8E0C5F025F0F0E58215827002158356
:060E5F00E0C838F0E822B3
:100E6500BB0110E58229F582E5833AF583E0F5F0CB
:100E7500A3E0225009E92582F886F008E622BBFEA8
:100E85000AE92582F8E2F5F008E222E5832AF583EE
:080E9500E993F5F0A3E99322B3
:0D0E9D00EF2BFFEE3AFEED39FDEC38FC22A4
:100EAA00E88FF0A4CC8BF0A42CFCE98EF0A42CFCE7
:100EBA008AF0EDA42CFCEA8EF0A4CDA8F08BF0A465
:100ECA002DCC3825F0FDE98FF0A42CCD35F0FCEBC4
:100EDA008EF0A4FEA9F0EB8FF0A4CFC5F02ECD3989
:0F0EEA00FEE43CFCEAA42DCE35F0FDE43CFC22F6
:100EF900EB9FF5F0EA9E42F0E99D42F0EC6480C870
:060F090064809845F0220F
:100F0F00EB9FF5F0EA9E42F0E99D42F0E89C45F038
:010F1F0022AF
:0C0F2000E0FCA3E0FDA3E0FEA3E0FF2244
:0C0F2C00E0F8A3E0F9A3E0FAA3E0FB2248
:100F38007401FF3395E0FEFDFCA3A3A3E02FFFF0AF
:100F4800E582158270021583E03EFEF0E582158287
:100F580070021583E03DFDF0E5821582700215836D
:050F6800E03CFCF0225A
:0C0F6D00ECF0A3EDF0A3EEF0A3EFF022F7
:100F7900A8828583F0D083D082120F90120F90122D
:100F89000F90120F90E473E493A3C583C5F0C58352
:100F9900C8C582C8F0A3C583C5F0C583C8C582C8C2
:010FA9002225
:0C0FAA00A42582F582E5F03583F5832252
:100FB600FAE6FB0808E6F925F0F618E6CA3AF6223C
:090FC600E0FBA3E0FAA3E0F9222C
:100FCF00F8E0FBA3A3E0F925F0F0E58215827002AB
:070FDF001583E0FA38F0224F
:090FE600EBF0A3EAF0A3E9F0220C
:0C0FEF00E493FB740193FA740293F9225E
:100FFB00BB010789828A83020FC65005E9F80210EC
:10100B00C2BBFE05E9F80210D489828A83020FEF76
:10101B00BB011A89828A83D0F0D0E0F8D0E0F9D0F6
:10102B00E0FAD0E0FBE8C0E0C0F0020FE65016E9B2
:10103B00F8D083D082D0E0F9D0E0FAD0E0FBC082C8
:10104B00C0830210CBBBFE16E9F8D083D082D0E070
:0F105B00F9D0E0FAD0E0FBC082C0830210DD22A2
:10106A00D083D082F8E4937012740193700DA3A315
:10107A0093F8740193F5828883E473740293686029
:06108A00EFA3A3A380DF29
:061090008A838982E473EB
:1010E600E5192462F582E43402F583E005192290BD
:1010F600025F300703900262E475F001120FCF021F
:101106000D9D2000E97F2ED2008018EF540F249009
:10111600D43440D4FF30040BEF24BFB41A0050037C
:101126002461FFE51A6002151A051DE51D7002050A
:101136001C30070E90025FE475F001120FCFEF022C
:101146000E050243AD7403D2078003E4C207F51906
:1011560090025F120FE6E4F51AF51CF51DE51A601C
:10116600077F2012112980F5751BFFC201C200C23C
:1011760002C203C205C206C2081210F5FF700D3086
:1011860007057F0012113AAF1DAE1C22B4255FC2BF
:10119600D5C2041210F5FF24D0B40A00501A75F017
:1011A6000A781A30D50508B6FF0106C6A426F62029
:1011B600D5047002D20380D924CFB41A00EF5004AC
:1011C600C2E5D20402133BD20180C6D20080C0D24F
:1011D6000280BCD2D580BAD20580B47F20121129F4
:1011E6002002077401B51A0040F11210E6FF121131
:1011F60029021163D208D20680951210E6FB12105E
:10120600E6FA1210E6F94A4B7006790C7A147BFF5F
:1012160020022EE51A602A7E008E82758300120D4A
:10122600B660060EEE651B70F0C2D5EBC0E0EAC0F4
:10123600E0E9C0E0EE121382D0E0F9D0E0FAD0E0A7
:10124600FB120D9DFF60AAEBC0E0EAC0E0E9C0E03A
:10125600121129D0E02401F9D0E03400FAD0E0FBE5
:10126600E51B0460DCD51BD980877BFF7A13797E6A
:10127600D202809C791080027908C206C2088008D2
:10128600D2D5790A8004790AC2D5E51B047002F525
:101296001BE4FAFDFEFF1210E6FC7B082001131288
:1012A60010E6FD7B1030000A1210E6FE1210E6FF73
:1012B6007B20EC3382D592D55013C3E43000069FD1
:1012C600FFE49EFEE42001039DFDE49CFCE4CBF8D4
:1012D600C201EC700CCFCECDCCE824F8F870F380C8
:1012E60017C3EF33FFEE33FEED33FDEC33FCEB3388
:1012F600FB994002FB0FD8E9EB300105F8D0E0C4BA
:1013060048B201C0E00AEC4D4E4F78207B0070C217
:10131600EAB51B0040BCC0E0121384D0F0D0E02038
:101326000104C4C0E0C4B201C0F0121112D0F0D55D
:10133600F0EB02116312106A120053127A5811D19F
:101346004C11CD42127E4F12864412864911E64355
:08135600128C55127046127052
:10135E0045127047142C5011D52D11D92E11FC2B7E
:10136E0011DD2311FA2014152A119548000011F4ED
:10137E003F3F3F00790AA2D5200314300509B9106A
:10138E00020404B9080104A2D5200602500104206B
:10139E0002689202B51A005034C0E07F2030031963
:1013AE007F30A20272067205500F1213DBC202C208
:1013BE0006C205C2087F30800F300503E9C0E01277
:1013CE001129300503D0E0F9D0E0B51ACC3005175D
:1013DE007F30B9100C1211297F583004077F7880A6
:1013EE0003B908031211293002057F2D0211297F3E
:1013FE00202008F87F2B2006F322920280CF286E41
:10140E00756C6C2900D2011210E63001F8C2017819
:10141E001A30D50108F60211952D50434958121075
:10142E00E62403B405004001E49014279312111A28
:0D143E00743A12111AD203751A0402127AC0
:10109600EF4E6012EF60010EEDBB010B89828A8371
:1010A600F0A3DFFCDEFA2289F05007F709DFFCA97E
:0C10B600F022BBFEFCF309DFFCA9F022D5
:0910C200E6FB08E6FA08E6F92253
:0910CB00EBF608EAF608E9F6224A
:0910D400E2FB08E2FA08E2F9224D
:0910DD00EBF208EAF208E9F22244
:1043AD00EFB40A07740D1243B8740A309811A89926
:1043BD00B8130CC2983098FDA899C298B811F63070
:0743CD0099FDC299F5992248
:00000001FF
